:100000000C94E7000C940F010C940F010C940F0159
:100010000C940F010C940F010C940F010C94B21569
:100020000C940F010C940F010C940F010C94F41715
:100030000C940F010C948D170C940F010C940F016C
:100040000C9470150C940F010C940F010C940F017B
:100050000C940F010C940F010C940F010C940F01E0
:100060000C946E160C940F01000000002400270071
:100070002A0000000000250028002B0000000000DE
:1000800023002600290004040404040404040202DA
:100090000202020203030303030302020301020438
:1000A00008102040800102040810200102040810FA
:1000B0002040804000000009000302000004050801
:1000C000000000000000000000000097A0895B5ABB
:1000D0000F830DC95F6035C2E907E18C24671E45B7
:1000E0008E086325F0150A17BE0694F778EA4B00D0
:1000F0001AC53E5EFCDBCB75230B2039B12158EDD0
:10010000953857AE147D88ABA844AF4AA547868B77
:10011000301BA64D929EE7536FE57A3CD385E6DC13
:10012000695C29372EF528F4668F3641193FA10105
:10013000D85049D14C84BBD05912A9C8C487827405
:10014000BC9F56A4646DC6ADBA034034D9E2FA7CB4
:100150007B05CA2693767EFF5255D4CFCE3BE32F44
:10016000103A11B6BD1C2ADFB7AAD577F898022C31
:100170009AA346DD99659BA72BAC09811627FD1331
:10018000626C6E4F71E0E8B2B97068DAF661E4FB58
:1001900022F2C1EED2900CBFB3A2F1513391EBF930
:1001A0000EEF6B31C0D61FB5C76A9DB854CCB07383
:1001B00079322D7F0496FE8AECCD5DDE72431D18E8
:1001C00048F38D80C34E42D73D9CB497311811241B
:1001D0001FBECFEFD8E0DEBFCDBF11E0A0E0B1E0A1
:1001E000E0ECF6E502C005900D92A634B107D9F710
:1001F00023E0A6E4B1E001C01D92A839B207E1F7FF
:1002000010E0C7EED0E004C02197FE010E94532BFE
:10021000C63ED107C9F70E9458180C945E2B0C9467
:100220000000000000000000000000008BE290E0F1
:100230000197F1F708959091A0029111FCCF91E000
:100240009093A00240939F022FEF20939E02109262
:100250009D02260F20939C0290939B0290919B02FB
:10026000880F892B80939B0280919A028130F9F448
:1002700010929A0280919B028093BB008091BC00F7
:1002800083FDF8CF85EC8093BC008091A002813083
:10029000E1F380919D02861710F460919D02AAE718
:1002A000B2E0EAE5F2E080E0861303C0089585EE4F
:1002B000EACF9D9191938F5FF7CF982F20915902AC
:1002C00081E0213208F043C08091A0028111FCCF6F
:1002D0008091580232E03093A00290939F029FEFEA
:1002E00090939E0210929D0220939C02A8E3B2E09C
:1002F000EAE7F2E090E0291331C010929B0290915E
:100300009B02880F892B80939B0280919A028130F7
:1003100049F510929A0280919B028093BB008091D4
:10032000BC0083FDF8CF85EC8093BC008091A002D7
:100330008230E1F380919E028F3FB1F080919E0266
:100340008032A1F080919E02803391F084E010927F
:100350003702109259021092360208953D9131935E
:100360009F5FC9CF85EEE0CF80E0F1CF82E0EFCF95
:1003700083E0EDCF0895089580E991E008958430F9
:1003800081F028F48230E9F08330F9F00895883064
:1003900071F0893091F08530B9F4809180008F7DC3
:1003A00003C0809180008F778093800008958091B2
:1003B000B0008F778093B00008958091B0008F7D5A
:1003C000F9CF84B58F7784BD089584B58F7DFBCF39
:1003D000CF93DF93282F30E0F901EC54FF4F849145
:1003E000F901E356FF4FD491F901EA57FF4FC49149
:1003F000CC23A1F081110E94BF01EC2FF0E0EE0FA1
:10040000FF1FE458FF4FA591B491EC91ED2381E0DB
:1004100090E009F480E0DF91CF91089580E090E0D2
:10042000FACF1F93CF93DF93282F30E0F901EC54DC
:10043000FF4F8491F901E356FF4FD491F901EA5738
:10044000FF4FC491CC23A9F0162F81110E94BF0148
:10045000EC2FF0E0EE0FFF1FEE58FF4FA591B49187
:100460008FB7F894EC91111108C0D095DE23DC937E
:100470008FBFDF91CF911F910895DE2BF8CF10929F
:1004800035021092340210923702109259021092E3
:10049000A00281E080939F0210929A0261E082E1C3
:1004A0000E94110261E083E10E941102E9EBF0E099
:1004B00080818E7F808380818D7F80838CE5809397
:1004C000B80085E48093BC008AEB91E090933302FE
:1004D000809332028BEB91E0909331028093300253
:1004E0000895CF93DF9390E0FC01E356FF4F2491F2
:1004F0008A579F4FFC0184918823D1F090E0880FA8
:10050000991FFC01E859FF4FA591B491FC01EE58E9
:10051000FF4FC591D49161110EC09FB7F8948C9193
:10052000E22FE0958E238C932881E223E8839FBFFE
:10053000DF91CF9108958FB7F894EC91E22BEC9373
:100540008FBFF6CFCF92DF92EF92FF926FB7F89402
:100550008091900190919101A0919201B0919301AD
:1005600050918F0126B535B3432F417030FF04C041
:1005700041E02F3F09F440E06FBF6C017D0137E09F
:10058000CC0CDD1CEE1CFF1C3A95D1F7C50ED11C1E
:10059000E11CF11CC81AD90AEA0AFB0A880F991F44
:1005A000AA1FBB1FC81AD90AEA0AFB0A63E0CC0CCF
:1005B000DD1CEE1CFF1C6A95D1F730E0A3E3B3E02D
:1005C0000E948528672F782F892F99276C0D7D1D14
:1005D0008E1D9F1D442321F06D5C7C4F8F4F9F4FDC
:1005E000FF90EF90DF90CF9008958F929F92AF92FF
:1005F000BF92CF92DF92EF92FF924B015C010E947B
:10060000A2026B017C010E94A2026C197D098E0975
:100610009F09683E734081059105A8F321E0821A85
:100620009108A108B10888EEC80E83E0D81EE11C2D
:10063000F11C81149104A104B10429F7FF90EF90FB
:10064000DF90CF90BF90AF909F908F9008952FB77D
:10065000F894609190017091910180919201909134
:1006600093012FBF08954F925F926F927F929F9256
:10067000AF92BF92CF92DF92EF92FF920F931F93B0
:10068000CF93DF9300D01F92CDB7DEB7F090AD02CD
:100690008091B0029091B102A091B202B091B302E8
:1006A000892B8A2B8B2BD9F00E94A2020091A902E0
:1006B0001091AA022091AB023091AC02601B710B29
:1006C000820B930B0091B0021091B1022091B20203
:1006D0003091B3026017710782079307C8F20E9436
:1006E000A2026093A9027093AA028093AB02909336
:1006F000AC02E091B802F091B902309759F0409104
:10070000B4025091B5026091B6027091B7028F2D7C
:100710000995F82E0091A7021091A8024F2C512C98
:10072000712C612C0115110509F45EC0D8011C96CD
:10073000EC901C978091AE029091AF0284369105A7
:1007400010F41C961C92D801ED91FC91A280B3800C
:1007500019821A821B82FF2089F1F8013696D12C6A
:10076000C12C2191222319F19280992001F130E0CE
:1007700050E040E02F5F3F4F4F4F5F4FC301B2014A
:100780000E94D22A9B01AC01892D90E0B0E0A0E04C
:10079000BC01CD016F5F7F4F8F4F9F4F0E94D22AC8
:1007A000A1E0B0E0AC0FBD1FAC0DBD1D8C93BFEF41
:1007B000CB1ADB0A83E0C816D10499F6D8011D963E
:1007C0004D915C911E9712966D917C919E012F5FC9
:1007D0003F4FC801F5010995D8011C96EC921C9772
:1007E00014960D911C919ECF8091A5029091A60226
:1007F0008C010F5F1F4F1093A6020093A50249972B
:10080000B4F10E942703C090A102D090A202E09010
:10081000A302F090A4029B01AC012C193D094E09E2
:100820005F0921F421E030E040E050E088EE93E001
:10083000089FB001099F700D189F700D1124072E9D
:10084000000C880B990B0E9463283093AF02209311
:10085000AE021092A6021092A5020E942703609396
:10086000A1027093A2028093A3029093A4020F901E
:100870000F900F90DF91CF911F910F91FF90EF900C
:10088000DF90CF90BF90AF909F907F906F905F90E0
:100890004F900895282F382F37FD2095229F020E64
:1008A00020E0211D000C221F37FD20951124822FEE
:1008B00008951F93DC01FB017C9111964C911197D7
:1008C00012961C91972F990F990F990F35E5292FA3
:1008D000239F020E20E0211D1124822F672F6074B8
:1008E000572F507277FD6FC061115BC0511105C069
:1008F000922F9095892F90E004C025E5280F90E075
:100900008BEA4F3F09F424C0442309F47DC08823B7
:1009100031F0382F349F030E30E0311D832F222316
:1009200021F0249F020E20E0211D992331F0392F60
:10093000349F030E30E0311D932F1124342F309556
:10094000339F030E30E0311D1124830F230F930FCB
:100950001F3F09F421C030E0112321F0119F312DF8
:1009600009F03F5F332309F453C0882331F0482F47
:10097000439F040E40E0411D842F222321F0239F3A
:10098000020E20E0211D992331F0492F439F040ED0
:1009900040E0411D942F11248083218392831F9175
:1009A000089551110BC0392F2AEA329F030E30E00F
:1009B000311D11249BEA931B280F9CCF90E02095BA
:1009C000982F80E09ECF611112C051110CC0392FB9
:1009D0002AEA329F030E30E0311D11242BEA231B3B
:1009E00095E5930FEECF922F909520E08ACF51118D
:1009F00006C025E5280F9BEA981B822FF6CF2AEA2E
:100A0000280F90E0932FF8CF9FEF2FEF8FEFA0CF1D
:100A100090E020E080E0C0CFCF92DF92EF92FF9293
:100A2000CF93DF93EC01072E000C880B990B0E94EB
:100A3000B0296B017C0120E030E040E45FE30E94DC
:100A4000652A20E030E048E452E40E9406290E9432
:100A50007829C617D707D4F020E030E040EA5FE3FA
:100A6000C701B6010E94652A20E030E048E452E464
:100A70000E94062920E030E040E85FE30E949528CC
:100A80000E94782921E06C177D070CF420E0822F6A
:100A900090E0DF91CF91FF90EF90DF90CF9008959D
:100AA0008F929F92AF92BF92CF92DF92EF92FF927E
:100AB0000F931F93CF93DF93FC0120813181E0914D
:100AC0002C02F0912D0201E010E02E173F070CF0F0
:100AD00045C0D901AA0FBB1FE0912A02F0912B0259
:100AE000EA0FFB1FA080B18089010095109501706D
:100AF000112720FD27C02CE93FEFEA016B017C01A3
:100B00004901840E951EB401C5010E940C0521E027
:100B100030E0892BD1F48C0E9D1EB401C5010E94DA
:100B20000C0522E030E0892B81F4BE01680D791DAF
:100B3000C5010E940C0523E030E0892B31F40FEF52
:100B40001FEF0CC024E630E0D8CFF6018081918100
:100B500001968217930784F491838083C801DF9103
:100B6000CF911F910F91FF90EF90DF90CF90BF90AA
:100B7000AF909F908F90089511821082F70180812D
:100B800091810196E9CF85ED8093BC008091BC00F6
:100B900084FDFCCF1092A002089520916B01260FD6
:100BA0003327331F21323105ECF42091A002FC01E0
:100BB00090E080E0243069F082E00895A0916B011C
:100BC0002191AC01455B5E4FA40FB52FB11D2C9355
:100BD0000196861798F380916B01680F60936B0103
:100BE00080E0089581E00895ECEBF0E080818A7B5D
:100BF000808360E082E10E94110260E083E10C9456
:100C000011020895E091350280913402E81730F422
:100C1000F0E0E65AFD4F808190E008958FEF9FEF5E
:100C2000089590913502809134022FEF3FEF98178D
:100C300048F4E92FF0E0E65AFD4F208130E09F5F55
:100C400090933502C9010895809134029091350244
:100C5000891B990B0895CF92DF92EF92FF920F9329
:100C60001F93CF93DF937C01CB018A012091360241
:100C7000222389F0EB016B01C40ED51ECC15DD05D6
:100C800069F06991D701ED91FC910190F081E02D1F
:100C9000C7010995F3CF642F0E94CD05C801DF91EC
:100CA000CF911F910F91FF90EF90DF90CF9008951B
:100CB000CF93DF931F92CDB7DEB7698320913602C1
:100CC0002223F9F020915902203258F021E030E03F
:100CD000FC013383228390E080E00F90DF91CF917D
:100CE000089580913702E82FF0E0E85CFD4F99818C
:100CF00090838F5F809337028093590281E090E068
:100D0000ECCF61E0CE0101960E94CD05F7CFCF93E5
:100D1000DF93D1E0D093360288E680935802109298
:100D200037021092590260E08AEB92E00E94580666
:100D300060E88AEB92E00E94580680911A02CAE0AD
:100D40006C2F0E94E22A8295807F682F690F8AEBC0
:100D500092E00E94580680911B026C2F0E94E22AAA
:100D60008295807F682F690F8AEB92E00E94580677
:100D700080911C026C2F0E94E22A8295807F682F4E
:100D8000690F8AEB92E00E94580680911D026C2F39
:100D90000E94E22A8295807F682F690F8AEB92E099
:100DA0000E94580680911E026C2F0E94E22A8295B2
:100DB000807F682F690F8AEB92E00E94580680912D
:100DC0001F028E516C2F0E94E22A8295807F682F2D
:100DD000690F8AEB92E00E94580681E00E945D0153
:100DE00081111DC0D0933602109237021092590221
:100DF00060E08AEB92E00E945806809119026C2F05
:100E00000E94E22A8295807F682F690F8AEB92E028
:100E10000E94580681E00E945D0191E0811190E0FE
:100E2000892FDF91CF91089590E080E008950F938E
:100E30001F93CF93DF9320914A012F5F322F37709A
:100E400030934A0120FF2BC020E831FD206434702C
:100E500009F02062205FFC01EC01239600E011E024
:100E60006485662329F070E0C8010E94022B6F5F41
:100E70006187322F369F030E30E0311D112431116E
:100E800010C01682662311F0615061873196EC170D
:100E9000FD0731F7DF91CF911F910F91089520E069
:100EA000D4CF31503683EECF2F923F924F925F9244
:100EB0006F927F928F929F92AF92BF92CF92DF926A
:100EC000EF92FF920F931F93CF93DF9300D000D048
:100ED000CDB7DEB71C017C836B830E94A202D101D7
:100EE0001F962D913C91621B730B6A307105A8F31C
:100EF000F894AB81BC81ED91FC91119755B1506193
:100F000045B14F7E45B91996CC90199716968C919C
:100F1000BC2DB81B8B2FAB81BC8116968C9316977A
:100F20001F96BC901F9712962D913C9113973A8370
:100F300029831C966C911C971D967C911D971E967B
:100F4000DC901E976F5F7F5FD39417969C911797E5
:100F500018963C9118971A96AC901A971B96EC909D
:100F60001081A981BA8120E0F32E022F322F308127
:100F7000112788943111380F08F43FEF8195889438
:100F800060FD130F1795889461FD130F17958894D2
:100F900062FD130F1795889463FD130F17958894BE
:100FA00064FD130F1795889465FD130F17958894AA
:100FB00066FD130F1795889467FD130F1795889496
:100FC000232F6111212F8C0D122F002C55B900C039
:100FD000002C17FF45B931812227889400C000C03A
:100FE00000C000C045B93111390F00C000C0002C4D
:100FF00055B900C0002C16FF45B908F43FEF919594
:10100000889400C000C000C000C045B970FD230F27
:1010100000C000C0002C55B900C0002C15FF45B918
:101020002795889471FD230F00C000C000C000C048
:1010300045B92795889400C000C0002C55B900C060
:10104000002C14FF45B972FD230F2795889400C02A
:1010500000C000C000C045B973FD230F00C000C030
:10106000002C55B900C0002C13FF45B92795889472
:1010700074FD230F00C000C000C000C045B9279513
:10108000889400C000C0002C55B900C0002C12FF8D
:1010900045B975FD230F2795889400C000C000C096
:1010A00000C045B976FD230F00C000C0002C55B923
:1010B00000C0002C11FF45B92795889477FD230FB8
:1010C00000C000C000C000C045B92795889400C08A
:1010D00000C0002C55B900C0002C10FF45B9132FDB
:1010E0007111122F9A0D00C000C000C000C045B998
:1010F00000C000C000C0002C55B900C0002C17FF74
:1011000045B932812227889400C000C000C000C0C9
:1011100045B931113F0D00C000C0002C55B900C0C9
:10112000002C16FF45B908F43FEFEB0DF11D00C090
:1011300000C000C000C045B9D0FC230F00C000C0F3
:10114000002C55B900C0002C15FF45B9279588948F
:10115000D1FC230F00C000C000C000C045B92795D6
:10116000889400C000C0002C55B900C0002C14FFAA
:1011700045B9D2FC230F2795889400C000C000C059
:1011800000C045B9D3FC230F00C000C0002C55B9E6
:1011900000C0002C13FF45B927958894D4FC230F79
:1011A00000C000C000C000C045B92795889400C0A9
:1011B00000C0002C55B900C0002C12FF45B9D5FC69
:1011C000230F2795889400C000C000C000C045B917
:1011D000D6FC230F00C000C0002C55B900C0002C65
:1011E00011FF45B927958894D7FC230F00C000C094
:1011F00000C000C045B92795889400C000C0002CED
:1012000055B900C0002C10FF45B9132FD110122F73
:10121000F19400C000C000C000C045B9FE0C00C081
:1012200000C000C055B900C0002C17FF45B930817F
:101230002227889400C000C000C000C045B9311109
:10124000380F00C000C0002C55B900C0002C16FF9C
:1012500045B908F43FEF8195889400C000C000C0F4
:1012600000C045B960FD230F00C000C0002C55B977
:1012700000C0002C15FF45B92795889461FD230F08
:1012800000C000C000C000C045B92795889400C0C8
:1012900000C0002C55B900C0002C14FF45B962FDF8
:1012A000230F2795889400C000C000C000C045B936
:1012B00063FD230F00C000C0002C55B900C0002CF6
:1012C00013FF45B92795889464FD230F00C000C023
:1012D00000C000C045B92795889400C000C0002C0C
:1012E00055B900C0002C12FF45B965FD230F2795A5
:1012F000889400C000C000C000C045B966FD230F3F
:1013000000C000C0002C55B900C0002C11FF45B929
:101310002795889467FD230F00C000C000C000C05F
:1013200045B92795889400C000C0002C55B900C06D
:10133000002C10FF45B9132F6111122F8C0D00C026
:1013400000C000C000C045B900C0119709F03ECEF2
:1013500020E732E0A981BA810E94162B44E1442E95
:10136000512C612C712CA30192010E946328490128
:101370005A01F12CE12CB7018AE9A981BA81A89F11
:101380000A0E611DB89F600D711D11246B0F711D38
:1013900090E080E054E0660F771F881F991F5A95F0
:1013A000D1F7A30192010E943128DA01C901880D09
:1013B000991DAA1DBB1D893EE3E09E07A105B1054D
:1013C00008F434C0885E9340A109B10922E0B695C3
:1013D000A795979587952A95D1F727E0829F080EC4
:1013E000E11C929FE00CF11C1124E90EF11C2091EC
:1013F000490130E0820F931F8E0D9F1D4091900197
:10140000509191016091920170919301292F33279E
:10141000420F531F611D711D409390015093910124
:1014200060939201709393018093490178940E9494
:10143000A202D10150967C936E931F970F900F904C
:101440000F900F90DF91CF911F910F91FF90EF9030
:10145000DF90CF90BF90AF909F908F907F906F90D4
:101460005F904F903F902F900895249A08950F9386
:101470001F93CF93DF93CDB7DEB762970FB6F89483
:10148000DEBF0FBECDBF8C01F901DC011C968C9133
:101490007A8369835C834B835E834D8390819D87D0
:1014A00091819E8792819F878130F1F4CE010196D0
:1014B0000E94170783E0888B1A8A198AD801ED9158
:1014C000FC910484F585E02DBE016F5F7F4FC8015C
:1014D000099562960FB6F894DEBF0FBECDBFDF91BF
:1014E000CF911F910F9108951C861B861A8619862D
:1014F00018861F82DFCF0F931F93CF93DF93CDB753
:10150000DEB762970FB6F894DEBF0FBECDBF8C0179
:10151000F901DC011C968C917A8369835C834B838F
:101520005E834D8390819D8791819E8792819F8765
:101530008130E9F4CE0101960E941707188A1A8AB1
:10154000198AD801ED91FC910484F585E02DBE0146
:101550006F5F7F4FC801099562960FB6F894DEBFA2
:101560000FBECDBFDF91CF911F910F9108951C86C3
:101570001B861A86198618861F82E0CF10921002E9
:101580001092110210921202109213021092FF0197
:1015900010920002109201021092020208951F930D
:1015A000CF93DF939091EA01913079F410E0C82F46
:1015B000D0E0CD5FDD4F188364E170E080E090E023
:1015C0000E94F5021F5F1A30B1F7DF91CF911F9192
:1015D0000895CF93C1E361E08BE00E9411020E9465
:1015E000110160E08BE00E9411020E941101C150C4
:1015F00091F7CF910895CF938A30D0F4E82FF0E09F
:10160000E95FFE4FC0816C2F687085E00E94110277
:101610006C2F647086E00E9411026C2F627087E06C
:101620000E9411026C2F617088E0CF910C9411021E
:1016300061E085E00E94110261E086E00E941102F3
:1016400061E087E00E94110261E0EECF0F931F93EB
:10165000CF93DF9300D01F92CDB7DEB71092AD02CB
:101660000FEC11E019821A821B82B801CE0101969B
:101670000E9459040D5F1F4F81E0043E180791F747
:101680000E9433030F900F900F90DF91CF911F9125
:101690000F9108958F929F92AF92BF92CF92DF9257
:1016A000EF92FF920F931F93CF93DF93982EC62F45
:1016B000842F822E6AE00E94E22A5C01C12CD12C88
:1016C0007601D0E0CD5FDD4F8E010F5F1F4F892D7A
:1016D0000E94E801892B59F48FEFC81AD80AE80A4A
:1016E000F80A8820A1F3A882F801B082F0CF81E047
:1016F000F9EECF16F3E0DF06E104F1040CF480E02C
:10170000DF91CF911F910F91FF90EF90DF90CF90DD
:10171000BF90AF909F908F900895CF93DF93EB0190
:1017200091E09093360291E1909358021092370223
:1017300010925902682F8AEB92E00E9458066D2F92
:101740008AEB92E00E9458066C2F8AEB92E00E948E
:10175000580681E0DF91CF910C945D01CF93DF9328
:10176000EC010E943F02BE016656734086E0660FA0
:10177000771F8A95E1F77093B2016093B1016061C0
:1017800083E00E948D0BDF91CF910C94F40581E0F2
:1017900090EC9093B4018093B30161E070EC82E02F
:1017A0000E948D0B6091000170910101665673409B
:1017B00086E0660F771F8A95E1F77093B201609318
:1017C000B101606183E00C948D0B81E090E890930F
:1017D000B4018093B30161E070E882E00E948D0B58
:1017E00081E080934601089590E080E00895FC0137
:1017F000858596850895CF93DF9300D000D000D0E3
:10180000CDB7DEB7AB011C821D821E82DC01ED91DB
:10181000FC910190F081E02D19821A821B829E01B9
:101820002F5F3F4FBE016C5F7F4F099526960FB625
:10183000F894DEBF0FBECDBFDF91CF910895CF9357
:1018400081E08093360288E6809358021092370236
:101850001092590260E08AEB92E00E94580681E003
:101860000E945D01811169C041E067E088E60E9445
:101870001B011092350280933402873008F45DC05A
:101880008AEB92E00E941106982F92959770CAE019
:101890008F709C9F800D1124809319028AEB92E037
:1018A0000E941106982F92959F708F709C9F800DBB
:1018B000112480931A028AEB92E00E941106982F5D
:1018C000929593708F709C9F800D112480931B02C2
:1018D0008AEB92E00E941106982F92959F708F706C
:1018E0009C9F800D112480931C028AEB92E00E9441
:1018F0001106982F92959F708F709C9F800D1124D8
:1019000080931D028AEB92E00E941106982F929517
:101910009F708F709C9F800D112480931E028AEB14
:1019200092E00E941106982F9F70925E82958F70B0
:101930008C9F900D112490931F0280911902809327
:10194000FC0180911A028093FA0180911B0280931E
:10195000F90180911D0224E6622F0E94E22A9093F1
:101960000F0280911E020E94E22A9093FE01809154
:101970001F0290E08E54984F64E670E00E94022BA4
:101980008093FD01CF910895CF93DF9381E0809301
:10199000360281E180935802109237021092590268
:1019A00065E08AEB92E00E94580680E00E945D01AB
:1019B00041E062E081E10E941B01109235028093B8
:1019C00034028AEB92E00E941106D82F80E0C82FE3
:1019D0008AEB92E00E9411068C2B9D2BDF91CF9118
:1019E0000895CF93C82F0E94C40C807FBC016C2B3C
:1019F0007093B0016093AF0185E0CF910C948D0B93
:101A00002F923F924F925F926F927F928F929F920E
:101A1000AF92BF92CF92DF92EF92FF920F931F93FC
:101A2000CF93DF9300D000D000D0CDB7DEB78DECE0
:101A300092E090932B0280932A028091CA0290E058
:101A400090932D0280932C028091970390E09093C5
:101A50002F0280932E028091C602853009F04DC07E
:101A60008091CF029091D002885891098D359105CF
:101A700008F073C08091CA02843009F042C080919E
:101A8000D1029091D20280974797D8F58091D302E6
:101A90009091D40209970997A0F51092290210920B
:101AA00028028FEF9FEFDC018093240290932502A0
:101AB000A0932602B093270283E090E09093210246
:101AC000809320028091C101882309F433C61092CB
:101AD000C1011092F70180E00E94F10C0E94E50B19
:101AE00068EE73E080E090E00E94F5020E941F0C17
:101AF00082E08093C6021092CA02C12CD12C7601DA
:101B000028C68091CA02843440F18091D10290911C
:101B1000D202825491098E9700F530E020E080E0F7
:101B200090E0DC01F901ED52FD4F408151814950B7
:101B300051094930510588F4F901EB52FD4F4081BC
:101B40005181475151094231510528F1408151815C
:101B5000465051094730510580F18091CA028A31BF
:101B600008F45FC08091CD029091CE02843F9140F5
:101B700048F510922902109228028FEF9FEFDC01A6
:101B80008093240290932502A0932602B09327020B
:101B90008BE090E093CF880F991FAA1FBB1F816035
:101BA0002C5F3F4F2038310509F0BCCF20E230E0F8
:101BB000309329022093280277CF880F991FAA1FFC
:101BC000BB1FEECF8091CF029091D00285974B97AB
:101BD00040F5E6ECF2E082E090E040E050E0BA014F
:101BE000DC0111962091CA022A171B0609F00CF499
:101BF000F3C023853485275031092730310508F09B
:101C0000EAC025853685235131092F30310508F486
:101C1000D5C0258536852A5031092930310508F48B
:101C2000D5C08091CA028A31F0F18091CD029091A5
:101C3000CE028032934008F49CCF8091CF029091E5
:101C4000D002C697869778F58091D1029091D20202
:101C5000C697869740F5E6ECF2E083E090E040E03E
:101C600050E0BA01DC0111962091CA022A171B0626
:101C700009F00CF4D8C0258536852C5031092B305D
:101C8000310508F0CFC027853089255231092B3125
:101C9000310508F4BAC0278530892C5031092A3023
:101CA000310508F4BAC08091CA02823238F18091BD
:101CB000CF029091D0020697079700F5E6ECF2E08C
:101CC00082E090E040E050E0BA01DC011196209102
:101CD000CA022A171B0609F00CF4D1C023853485EB
:101CE0002E5131092731310508F4B4C023853485DC
:101CF0002C5031092B30310508F4BBC01C821B82EB
:101D000081E090E09A8389838091CA028D3008F443
:101D1000E7C049E753E0BE016D5F7F4FCE010196FA
:101D20000E945005892B09F0DBC049E753E0BE0152
:101D30006D5F7F4FCE0101960E945005019709F01B
:101D4000CFC049E753E0BE016D5F7F4FCE010196E2
:101D50000E9450058C01892B09F0C2C0C12CD12CE6
:101D600076012091CA0289819A812817190609F003
:101D70000CF4A7C049E753E0BE016D5F7F4FCE0171
:101D800001960E9450055C0149E753E0BE016D5F7A
:101D90007F4FCE0101960E945005B1E0AB16B10411
:101DA00009F086C0892B09F09BC0CC0CDD1CEE1C11
:101DB000FF1C6894C0F80F5F1F4FD3CF440F551F0F
:101DC000661F771F4160029634960ACF440F551F55
:101DD000661F771FF8CFCD01019795958795909352
:101DE0002902809328020C972CF410922902109259
:101DF000280217CF409324025093250260932602B5
:101E00007093270284E090E059CE440F551F661F5F
:101E1000771F41600296349625CF440F551F661FE9
:101E2000771FF8CFCD01019795958795909329025B
:101E3000809328020C972CF4109229021092280209
:101E400032CF409324025093250260932602709370
:101E500027029ECE440F551F661F771F41602585C0
:101E600036853496235031092530310538F40296F1
:101E70002CCF440F551F661F771FF1CFCD0101975F
:101E800095958795909329028093280240972CF48A
:101E9000109229021092280231CF409324025093CD
:101EA000250260932602709327028CE090E006CE14
:101EB000AB28B1F40197A1F4CC0CDD1CEE1CFF1C87
:101EC0007ACF1093290200932802C0922402D09264
:101ED0002502E0922602F092270281E090E0EECD0A
:101EE0001C821B8281E090E09A83898380912C027E
:101EF00090912D02181619060CF07EC0E0912A026E
:101F0000F0912B0282E090E09A8389838281938111
:101F100089974E9708F070C083E090E09A83898398
:101F2000848195810B970A9708F066C04CEB51E0CD
:101F3000BE016D5F7F4FCE0101960E9450058C015E
:101F4000892B09F059C04CEB51E0BE016D5F7F4F0A
:101F5000CE0101960E945005019709F04DC0C12C99
:101F6000D12C760120912C0230912D0289819A8109
:101F7000821793070CF0E5C04CEB51E0BE016D5F9A
:101F80007F4FCE0101960E9450055C010330110580
:101F900039F14CEB51E0BE016D5F7F4FCE010196F0
:101FA0000E9450054C010330110561F44CEB51E0E7
:101FB000BE016D5F7F4FCE0101960E9450058816CD
:101FC0009906D1F4A114B10409F4AEC0AA94AB28C7
:101FD00099F4892889F4CC0CDD1CEE1CFF1CAEC0E2
:101FE0004CEB51E0BE016D5F7F4FCE0101960E9428
:101FF0005005A816B90669F2E0912A02F0912B0269
:1020000082819381C697869778F5848195814B97D5
:10201000459750F5DF0116967F0126ECE20EF11C84
:1020200020E030E040E050E060E070E080E090E0F0
:102030000D911C9111970950110908301105A0F458
:1020400012960D911C911397015111090D30110534
:1020500008F486C012960D911C9113970450110933
:102060000530110508F4A1C08091CA02893380F1BE
:1020700082819381895791098335910548F584813F
:102080009581CA97899720F59F012A5F3F4FC12C00
:10209000D12C760143E050E0D9016D917C911197EC
:1020A0006A5071096930710598F412966D917C91AE
:1020B0001397665171096131710508F47AC012965F
:1020C0006D917C91665071096730710508F4A0C06C
:1020D0008091CA02823209F0A0C0828193810A975E
:1020E000099708F09AC0A091CA02B0E0A150B04888
:1020F000AA0FBB1FAE0FBF1F8D919C910A97099726
:1021000008F08BC010922902109228028FEF9FEFE7
:10211000DC018093240290932502A0932602B093C1
:10212000270286E090E0CACC8A94892809F064CF1F
:10213000CC0CDD1CEE1CFF1C6894C0F80F5F1F4F19
:1021400011CF1093290200932802C0922402D0924A
:102150002502E0922602F092270282E090E0AECCC7
:1021600001E00E941D2B21601496AE15BF0509F0F9
:102170005FCF209324023093250240932602509390
:10218000270200E20E94382B209322023093230280
:1021900085E090E0909321028093200280E390E01C
:1021A00090932902809328028DCC01E00E941D2B80
:1021B000DBCFD701C601880F991FAA1FBB1F6C0177
:1021C0007D016894C0F84E5F5F4F2C5F3F4F4B33EB
:1021D000510509F061CF9F012A583F4FD9012D9138
:1021E0003C912A5031092930310508F071CF2CE19A
:1021F00030E03093290220932802C0922402D0922A
:102200002502E0922602F09227028AE090E056CC66
:10221000CC0CDD1CEE1CFF1CD6CF8281938189572C
:1022200091098335910560F58091CA02813240F1B0
:1022300084819581CA97899718F59F012A5F3F4F3E
:10224000C12CD12C760143E050E0D9016D917C91F5
:1022500011976A5071096930710590F412966D9169
:102260007C911397665171096131710598F112964D
:102270006D917C91665071096730710508F457C003
:10228000828193818C549109C59708F084C0809114
:10229000CA02843009F050C08481958180974797A5
:1022A00008F04AC0868197810997099708F044C0D1
:1022B00010922902109228028FEF9FEFDC01809389
:1022C000240290932502A0932602B093270287E070
:1022D00090E0F4CBD701C601880F991FAA1FBB1F3E
:1022E0006C017D016894C0F84E5F5F4F2C5F3F4FDB
:1022F0004332510509F0A9CF9F012A5B3F4FD90115
:102300002D913C912A5031092930310508F0B8CF80
:1023100020E130E03093290220932802C092240269
:10232000D0922502E0922602F0922702FACECC0C3F
:10233000DD1CEE1CFF1CD8CF8091CA02843458F1FA
:102340008481958189549109C39728F59F012A5F5B
:102350003F4FBF016A577F4FC12CD12C7601D90165
:102360004D915C911197495051094930510598F4AC
:1023700012964D915C911397465151094131510587
:1023800008F4A2C012964D915C9146505109473015
:10239000510508F4B8C08091CA028634C0F1828128
:1023A00093810C970B9798F58481958109970997EC
:1023B00070F5868197818C974F9748F58085918538
:1023C00089974D9720F59F01265F3F4FC12CD12C57
:1023D000760145E050E0D9016D917C9111976C50E8
:1023E00071096B30710598F412966D917C91139779
:1023F0006E5171096731710508F48AC012966D91AA
:102400007C91695071096930710508F4B0C0809100
:10241000CA02883508F4BAC082819381855891092F
:102420008B35910508F0B2C0848195818254910961
:102430008E9708F0ABC08F01045C1F4F8DE190E0D8
:1024400030E020E04091CA024450550B84179507B4
:1024500014F5A80142505109DA014D915C9149509F
:1024600051094830510508F091C0BC016F5F7F4FA2
:10247000D8014D915C911197475051094730510552
:1024800008F47AC04D915C9148515109423151058F
:1024900008F479C0CB01019795958795909329020F
:1024A000809328028A970CF471C0C901330FAA0BDC
:1024B000BB0B8093240290932502A0932602B09335
:1024C000270289E090E0FACAD701C601880F991F58
:1024D000AA1FBB1F6C017D016894C0F82C5F3F4FA1
:1024E0006217730709F03BCF20E230E030932902F6
:1024F00020932802C0922402D0922502E092260264
:10250000F0922702E4CECC0CDD1CEE1CFF1CE6CFC3
:10251000D701C601880F991FAA1FBB1F6C017D013F
:102520006894C0F84E5F5F4F2C5F3F4F45345105B4
:1025300009F051CF9F0126573F4FD9012D913C9172
:102540002C5031092B30310508F061CF20E230E00A
:102550003093290220932802C0922402D0922502AF
:10256000E0922602F092270288E090E0A7CACC0C05
:10257000DD1CEE1CFF1CD6CF220F331F21600296FC
:102580000C5F1F4F5FCF220F331FF9CF8091CA021C
:10259000803279F5828193810697069750F5848180
:1025A00095810997099728F59F012A5F3F4FBF0141
:1025B000625C7F4FC12CD12C7601D9014D915C9189
:1025C0001197465051094630510598F412964D9195
:1025D0005C911397495151094331510508F484C066
:1025E00012964D915C91495051094930510508F4BA
:1025F0009CC080912C0290912D029E838D83069722
:102600000CF476CA8F010E5F1F4F85ECC82E8DE942
:10261000D82E8CE1E82E81E8F82E93E0292E312C7B
:10262000D80114966D917C911597AD90BC9090E077
:1026300080E00E94AE292B013C01B50190E080E0D2
:102640000E94AE294B015C012DEC3CEC4CE45FE3B5
:102650000E94652A9B01AC01C301B2010E940129BD
:10266000F0E0E0E087FD14C02DEC3CEC4CE45FE3CF
:10267000C301B2010E94652A9B01AC01C501B401EE
:102680000E940129E2E0F0E087FD02C0E1E0F0E015
:10269000A701960163E971E080E091E00E94D22AEF
:1026A0006F01FF0FEE08FF08C626D726E826F92699
:1026B000BFEF2B1A3B0A0E5F1F4FED81FE81E21523
:1026C000F30509F0ADCFC0922402D0922502E0922A
:1026D0002602F092270280E290E0909329028093F4
:1026E00028028FEF9FEFEAC9D701C601880F991F13
:1026F000AA1FBB1F6C017D016894C0F82C5F3F4F7F
:102700006217730709F059CF2EE030E030932902A9
:1027100020932802C0922402D0922502E092260241
:10272000F09227028FE090E0C9C9CC0CDD1CEE1CB2
:10273000FF1CE4CFC0902402D0902502E090260236
:10274000F090270282E08093C6021092CA020E9493
:10275000E90AC701B60126960FB6F894DEBF0FBE90
:10276000CDBFDF91CF911F910F91FF90EF90DF9040
:10277000CF90BF90AF909F908F907F906F905F9021
:102780004F903F902F9008954F925F926F927F925B
:10279000AF92BF92CF92DF92EF92FF920F931F936F
:1027A000CF93DF938AE08093030280930402E09149
:1027B0000001F0910101CF0168EE73E00E94EE2A62
:1027C000CB012AE030E0B9010E94EE2AC82F8093A5
:1027D0000502CF0164E670E00E94EE2ACB01B90148
:1027E0000E94EE2A80930602CF01B9010E94EE2AD0
:1027F000482FCB01B9010E94EE2A80930702409333
:1028000008020E94BE0AD2E0B12C8AE0A82E0E94E3
:10281000000D6B017C01C0921502D0921602E0926D
:102820001702F09218020E9427030D2F10E040902B
:1028300010025090110260901202709013026419FD
:10284000750986099709643671058105910570F04F
:102850000E9427036093100270931102809312026A
:1028600090931302F801ED5FFD4FC0830E94270390
:102870004090FF01509000026090010270900202AF
:102880006419750986099709683C710581059105E8
:1028900070F00E9427036093FF0170930002809301
:1028A000010290930202F801ED5FFD4FA0822DEF2F
:1028B000C21622E0D2062FEFE206F10409F057C05B
:1028C0000E941F0CF801ED5FFD4FC08320910502AF
:1028D0004AE08091060290E0249F800D911D112412
:1028E000489FB001499F700D112420910702260FC7
:1028F000372F311D429FB001439F700D11248091ED
:102900000802860F972F911D893324E0920760F506
:102910009093010180930001809100019091010149
:102920008B36934030F48BE693E0909301018093D3
:10293000000180910001909101010E94AE0B0E9464
:10294000C70B81E08093F8018B2DDF91CF911F9110
:102950000F91FF90EF90DF90CF90BF90AF907F905E
:102960006F905F904F90089588E394E0D1CF8DED04
:10297000C81682E2D8068FEFE806F10481F4F80168
:10298000ED5FFD4FC083D150D13009F4D5E0ED2F7C
:10299000F0E0ED5FFD4FC0810E94BE0A38CF2DE30D
:1029A000C21622ECD2062FEFE206F10449F4F80138
:1029B000ED5FFD4FC083DF5FD63049F7D2E0E7CF50
:1029C0008DE9C81682E6D8068FEFE806F10471F4A7
:1029D000CF5FD23039F4C23038F40E94BE0ABB2433
:1029E000B39415CFCA30C8F3C0E0F7CF27E5C216BD
:1029F00028EAD2062FEFE206F10409F008CFC15011
:102A0000D23021F4CA3048F3C1E0E7CFCA3028F30E
:102A1000C9E0E3CF80914601882341F00E94C70BB3
:102A200080E00E94F10C1092460108958091F70118
:102A30008F5F8D3030F48093F7018091F7010C9413
:102A4000F10C8CE0F8CF1F93CF93DF93C82FD62FD4
:102A5000142F8091E601882331F10E94A82722E3F8
:102A600030E040E050E00E943128609348010E942D
:102A7000A8272CE231E040E050E00E9431286A3281
:102A800071408105910579F4E0914801E63058F4F0
:102A9000F0E0ED5FFD4F8AE0808362E370E080E06C
:102AA00090E00E94F5022AE0812F622F0E94E22A24
:102AB00090930802809307028D2F0E94E22A909340
:102AC0000602809305028C2F0E94E22A9093040252
:102AD00080930302DF91CF911F9108950E94592B9B
:102AE0001F920F920FB60F9211244F935F936F9323
:102AF0007F938F939F9340919001509191016091AA
:102B000092017091930180918F0190918E01943088
:102B100019F510928E0190918E0190FD21C08A5975
:102B20008D3728F08D574F5F5F4F6F4F7F4F8093EA
:102B30008F014093900150939101609392017093A3
:102B400093019F918F917F916F915F914F910F9022
:102B50000FBE0F901F9018959F5F90938E01DBCF53
:102B60008959DECF1F920F920FB60F9211242F9327
:102B70003F934F935F936F937F938F939F93AF9305
:102B8000BF93EF93FF938091C7020E94E8012091C9
:102B9000CB023091CC022F5F3F4F3093CC02209379
:102BA000CB029091CA02953618F096E09093C60237
:102BB0009091C602943009F466C0B8F49230F1F0F6
:102BC000933009F444C09091C902992309F46BC071
:102BD00081117AC08091C802882309F463C0809172
:102BE000C80261E00E9411025EC0953009F457C02E
:102BF000963049F791E0909397034FC08111E3CF4E
:102C00002091CB023091CC022436310528F4109269
:102C1000CC021092CB02D7CF109297031092CA0227
:102C20002091CB023091CC02E091CA0291E09E0F3C
:102C30009093CA02F0E0EE0FFF1FEA53FD4F30877A
:102C400027831092CC021092CB0293E019C08130FE
:102C500009F0B9CF2091CB023091CC02E091CA02A9
:102C600091E09E0F9093CA02F0E0EE0FFF1FEA532F
:102C7000FD4F308727831092CC021092CB0294E054
:102C80009093C602A0CF2091CB023091CC02882332
:102C900059F22536310508F496CF95E0F1CF811130
:102CA00092CFB5CF2D9AFF91EF91BF91AF919F91A8
:102CB0008F917F916F915F914F913F912F910F90E5
:102CC0000FBE0F901F9018958091C802882321F0A5
:102CD0008091C80260E086CF2D98E5CF1F920F92B9
:102CE0000FB60F9211242F933F934F935F936F93DF
:102CF0007F938F939F93AF93BF93EF93FF938091B5
:102D0000B900887F803609F44AC0F0F5883209F4AA
:102D1000A7C018F5803109F49BC0B8F4882309F4E2
:102D2000F9C0883009F494C0FF91EF91BF91AF9141
:102D30009F918F917F916F915F914F913F912F91D3
:102D40000F900FBE0F901F901895883109F488C01E
:102D5000803251F780939E0214C0803409F49DC0E4
:102D600040F48033B9F38833F9F680939E0285EC02
:102D7000B0C0803509F485C0883509F496C0883420
:102D800099F60E94C305D0CF883909F48CC038F574
:102D9000883729F050F4883611F0803729F683E01F
:102DA0008093A00210928D0157C0883809F47BC02F
:102DB000803919F0803809F0B7CF80918D018032C9
:102DC00008F071C0E0918D0181E08E0F80938D013C
:102DD0008091BB00F0E0E359FE4F80833DC0803B13
:102DE00039F0E0F4803A09F479C0883A09F09CCFD0
:102DF00084E08093A00210926C0110926B01E0912C
:102E00003202F0913302099580916B0181110FC05C
:102E100081E080936B0110924B0109C0803C09F462
:102E2000A6CF883C09F4A3CF883B09F07DCFE09181
:102E30006C0181E08E0F80936C01F0E0E55BFE4F4A
:102E400080818093BB0090916C0180916B0129C0BF
:102E500080919B028093BB0085EC8093BC0064CF83
:102E600090919D0280919C02981758F5E0919D02E7
:102E700081E08E0F80939D02F0E0E658FD4F808147
:102E8000E9CFE0919D0281E08E0F80939D028091B9
:102E9000BB00F0E0E658FD4F808390919D02809149
:102EA0009C029817C8F285E8D8CFE0919D0281E096
:102EB0008E0F80939D028091BB00F0E0E658FD4F9D
:102EC000808380919F0281115CCF81E080939A0280
:102ED00084EA8093BC001092A00226CF85EC8093F8
:102EE000BC001092A00280918D01803230F4E091FC
:102EF0008D01F0E0E359FE4F108260918D0170E08A
:102F0000E0913002F09131028DE691E00995109246
:102F10008D010ACF10929E0234CF1F920F920FB6EE
:102F20000F9211242F933F934F935F936F937F934F
:102F30008F939F93AF93BF93CF93EF93FF93C091E2
:102F40004701C230C9F1E0F4CC2331F1C13069F15D
:102F5000CF5FC63008F045C0C0934701FF91EF91A5
:102F6000CF91BF91AF919F918F917F916F915F9121
:102F70004F913F912F910F900FBE0F901F9018957A
:102F8000C43041F100F1C53019F761E080E00E94E2
:102F900011028091030206C061E084E00E941102E8
:102FA000809108020E94FB0AD3CF61E083E00E9477
:102FB000110280910702F6CF61E081E10E941102C7
:102FC00080910602EFCF61E082E00E9411028091C1
:102FD0000502E8CF61E081E00E94110280910402C5
:102FE000E1CF10924701BACF1F920F920FB60F9206
:102FF00011242F933F934F935F936F937F938F93FE
:103000009F93AF93BF93EF93FF9360E083E00E94A1
:10301000110260E084E00E94110260E081E10E9400
:10302000110260E080E00E94110260E081E00E94F5
:10303000110260E082E00E9411028AE00E94FB0A15
:10304000FF91EF91BF91AF919F918F917F916F9180
:103050005F914F913F912F910F900FBE0F901F9056
:103060001895EDEAF2E08FEF8083128211821486C8
:1030700013868FEF9FEFDC0187839087A187B2874C
:103080000E943F02EAEBF2E01382128288EE93E0A4
:10309000A0E0B0E084839583A683B78387E391E0C3
:1030A00091838083E6ECF2E089E0818313820895C6
:1030B000CF93DF93CDB7DEB72E970FB6F894DEBF70
:1030C0000FBECDBF789484B5836084BD85B5836021
:1030D00085BD80916E00816080936E0082E0809358
:1030E00081008091810081608093810080918000C7
:1030F0008160809380008091B10084608093B100F2
:103100008091B00081608093B00087E880937A005E
:103110001092C10080E480937C0080917A008064EA
:1031200080937A0080917A0086FDFCCF80917800B0
:1031300060917900762F682F072E000C880B990B71
:10314000611571058105910511F00E94F7278091A5
:10315000A701811145C010929901109298018FEF3B
:1031600080939C0180939D0180939E0180939F0199
:103170008093A0018093A10181E08093A20110922D
:10318000A4011092A30110929B0110929A018091C8
:10319000A7029091A802892B31F486E991E09093DF
:1031A000A8028093A702E0919401F09195013097D5
:1031B00021F086E991E09583848386E991E09093FC
:1031C0009501809394011092A6011092A50185E2C9
:1031D00091E0909397018093960181E08093A701FD
:1031E000249A8FEC91E0909399018093980186E066
:1031F00090E09093A4018093A3018091B0029091FC
:10320000B102A091B202B091B302843C29E09207CE
:10321000A105B10520F484EC99E0A0E0B0E0809332
:10322000B0029093B102A093B202B093B3020E9495
:10323000260BF89482E08093B0008093B1009DE764
:103240009093B3001092B2008093700078948093B2
:10325000C6021092CA028091C70260E00E94710209
:103260000E943F0261E070EC82E00E948D0B81E0E1
:1032700090ED9093B4018093B30161E070ED82E032
:103280000E948D0B609100017091010166567340A0
:1032900036E0660F771F3A95E1F77093B2016093BD
:1032A000B101606183E00E948D0B0E94C40CBC01DF
:1032B000607F7093B0016093AF0185E00E948D0B39
:1032C0000E94F40560E08FE00E94710260E08EE0F1
:1032D0000E94710260E080E10E94710261E083E07F
:1032E0000E94710261E084E00E94710261E081E16C
:1032F0000E94710261E082E00E94710261E081E05F
:103300000E94710261E080E00E94710261E085E04C
:103310000E94710261E086E00E94710261E087E034
:103320000E94710261E088E00E94710261E08BE01E
:103330000E94710285E090E00E940028D82E8093C0
:10334000EA0184E090E00E940028E82E8093E901E1
:1033500083E090E00E940028F82E8093E80182E04C
:1033600090E00E940028082F8093E70181E090E020
:103370000E940028182F8093E50180E090E00E94D1
:1033800000288093E601823018F081E08093E60106
:1033900031E03D1518F481E08093EA0151E05E15BB
:1033A00018F481E08093E90161E06F1518F481E081
:1033B0008093E801023010F01092E701123010F013
:1033C0001092E50187E090E00E940028182F80937A
:1033D000E40186E090E00E9400288093E301183128
:1033E00018F099E09093E4018C3318F08EE180930B
:1033F000E30182E190E00E9408289093F601809317
:10340000F50180E190E00E9408289093F4018093F8
:10341000F3018EE090E00E9408289093F2018093DF
:10342000F1018CE090E00E9408289093F0018093D5
:10343000EF018AE090E00E9408289093EE018093CB
:10344000ED0188E090E00E9408289093EC018093C1
:10345000EB01F894109280001092810010926F009E
:103460008CED9FEF909389008093880083E0809398
:10347000800099E19093810080936F007894812C73
:10348000912C54018A940AE01AE080910201882369
:1034900041F00E941F0C0E94E50B0E94260B109227
:1034A00002010E94000D6B017C01C0921502D092B6
:1034B0001602E0921702F092180220E040E060E06D
:1034C0008FE00E944A0B811109C077ECC71678E3A0
:1034D000D7067FEFE706F10409F0ACC18091140232
:1034E000882309F46BC30E94BE0A9FE1F92EEE24E3
:1034F000E3940E94270340901002509011026090C4
:1035000012027090130264197509860997096436CE
:1035100071058105910598F00E94270360931002C0
:1035200070931102809312029093130280910F0204
:10353000602F0E94E22A90930402809303020E946B
:1035400027034090FF0150900002609001027090AC
:1035500002026419750986099709683C710581059D
:10356000910570F00E9427036093FF0170930002A1
:1035700080930102909302021093040210930302BD
:103580000E94000D6093150270931602809317023B
:1035900090931802673EE8E17E07EFEF8E079105F2
:1035A00069F480910F028F5F803218F480930F02CC
:1035B00002C0E0920F020E94BE0A9BCF653BFAE474
:1035C0007F07FFEF8F07910539F480910F0281503B
:1035D00069F7F0920F02EFCF673C78438F4F910568
:1035E00009F087CF80910F02602F0E94E22A90930A
:1035F0000402809303020E94BE0A8CE0F82EEE249F
:10360000E3940E94270340901002509011026090B2
:1036100012027090130264197509860997096436BD
:1036200071058105910598F00E94270360931002AF
:103630007093110280931202909313028091FE0105
:10364000602F0E94E22A90930602809305020E9456
:1036500027034090FF01509000026090010270909B
:1036600002026419750986099709683C710581058C
:10367000910570F00E9427036093FF017093000290
:1036800080930102909302021093060210930502A8
:103690000E94000D6093150270931602809317022A
:1036A00090931802673E38E173073FEF8307910557
:1036B00069F48091FE018F5F8D3018F48093FE01D4
:1036C00002C0E092FE010E94BE0A9BCF653B5AE415
:1036D00075075FEF8507910539F48091FE018150F0
:1036E00069F7F092FE01EFCF673C78438F4F910569
:1036F00009F087CF8091FE01602F0E94E22A90930B
:103700000602809305020E94BE0AA3E6FA2EB4E1E7
:10371000EB2E0E94270340901002509011026090FF
:1037200012027090130264197509860997096436AC
:1037300071058105910598F00E942703609310029E
:103740007093110280931202909313028091FD01F5
:10375000602F0E94E22A90930802809307020E9441
:1037600027034090FF01509000026090010270908A
:1037700002026419750986099709683C710581057B
:10378000910570F00E9427036093FF01709300027F
:103790008093010290930202109308021093070293
:1037A0000E94000D60931502709316028093170219
:1037B00090931802673EF8E17F07FFEF8F079105AE
:1037C00069F48091FD018F5F843618F48093FD01C8
:1037D00002C0E092FD010E94BE0A9BCF653B2AE435
:1037E00072072FEF8207910541F48091FD0181500E
:1037F000843160F7F092FD01EECF673C78438F4F44
:10380000910509F086CF2091FD01822F602F0E9443
:10381000E22A909308028093070280910F0280931E
:103820001D028091FE0180931E02225E20931F02E2
:103830000E9487068091150290911602A0911702AE
:10384000B0911802873938E693073FEFA307B10517
:1038500009F02EC38091F70181508093F7018D30DC
:1038600008F423C30E94E50B1092F7018091150222
:1038700090911602A0911702B09118028B3B9D41C6
:10388000A145B105C1F48091F3019091F4019093A9
:103890000101809300010E94C413609100017091A6
:1038A00001017093F4016093F301882321F080E11A
:1038B00090E00E941C288091150290911602A09120
:1038C0001702B09118028D31924EAF4FB105C1F47D
:1038D0008091F1019091F201909301018093000198
:1038E0000E94C41360910001709101017093F20174
:1038F0006093F101882321F08EE090E00E941C2863
:103900008091150290911602A0911702B0911802B1
:103910008D3D9242AF4FB105C1F48091EF0190917E
:10392000F00190930101809300010E94C413609103
:103930000001709101017093F0016093EF01882301
:1039400021F08CE090E00E941C288091150290915B
:103950001602A0911702B09118028D3F9240AF4F0E
:10396000B105C1F48091ED019091EE0190930101B8
:10397000809300010E94C4136091000170910101C5
:103980007093EE016093ED01882321F08AE090E0CE
:103990000E941C288091150290911602A091170296
:1039A000B09118028D33924CAF4FB105C1F48091A4
:1039B000EB019091EC0190930101809300010E9432
:1039C000C41360910001709101017093EC01609348
:1039D000EB01882321F088E090E00E941C28809170
:1039E000150290911602A0911702B0911802873E1D
:1039F0009841AF4FB10509F0B7C6FF24F394E090AA
:103A0000EA01E092080210930702F0920602109376
:103A1000050210930402109303020E94000D6093AC
:103A20001502709316028093170290931802673C58
:103A3000E8E37E07EFEF8E07910509F068C2F2E038
:103A4000DF2EEE24E394F090E901F0920802109347
:103A50000702D092060210930502109304021093FD
:103A600003020E94000D609315027093160280936A
:103A7000170290931802673C38E373073FEF830700
:103A8000910509F053C2E3E0DE2EEE24E394F090BA
:103A9000E801F092080210930702D09206021093F8
:103AA000050210930402109303020E94000D60931C
:103AB0001502709316028093170290931802673CC8
:103AC000E8E37E07EFEF8E07910509F03EC274E050
:103AD000D72EEE24E394F090E701F09208021093C1
:103AE0000702D0920602109305021093040210936D
:103AF00003020E94000D60931502709316028093DA
:103B0000170290931802673C38E373073FEF83076F
:103B1000910509F029C265E0D62EEE24E394F090D9
:103B2000E601F092080210930702D0920602109369
:103B3000050210930402109303020E94000D60938B
:103B40001502709316028093170290931802673C37
:103B5000E8E37E07EFEF8E07910509F014C256E007
:103B6000D52EEE24E394F090E501F0920802109334
:103B70000702D092060210930502109304021093DC
:103B800003020E94000D6093150270931602809349
:103B9000170290931802673C38E373073FEF8307DF
:103BA000910509F402C2673E78418F4F9105D9F61D
:103BB00061E0F612F7C11092E501D5CF1092FC0139
:103BC00081E08093FB0164E670E080E090E00E9479
:103BD000F50210920802109207028091FA01602FFC
:103BE0000E94E22A90930602809305020E94000D33
:103BF0006B017C01C0921502D0921602E09217026E
:103C0000F09218020E942703409010025090110277
:103C10006090120270901302641975098609970961
:103C2000643671058105910598F00E942703609321
:103C300010027093110280931202909313028091EC
:103C4000F901602F0E94E22A9093040280930302FC
:103C50000E9427034090FF015090000260900102F3
:103C6000709002026419750986099709683C71050C
:103C70008105910570F00E9427036093FF01709306
:103C800000028093010290930202109304021093A9
:103C900003027090F90121E0472D60E080E10E946D
:103CA0004A0B811108C057EEC51658E1D5065FEFE3
:103CB000E506F10449F481E0870D883108F0E7C09A
:103CC0008093F9010E94BE0A7090F90121E0472D0E
:103CD00060E08EE00E944A0B811108C065EBC616B9
:103CE0006AE4D6066FEFE606F10449F48FEF870D1C
:103CF000883108F0CFC08093F9010E94BE0A20E00D
:103D000040E060E08FE00E944A0B811109C087EC1F
:103D1000C81688E3D8068FEFE806F10409F059CFFA
:103D20000E94BE0A10920802109207028091F901C7
:103D3000602F0E94E22A90930402809303020E9463
:103D4000000D6B017C01C0921502D0921602E09228
:103D50001702F09218020E94270340901002509020
:103D6000110260901202709013026419750986099D
:103D70009709643671058105910598F00E94270323
:103D800060931002709311028093120290931302B9
:103D90008091FA01602F0E94E22A9093060280939C
:103DA00005020E9427034090FF015090000260909E
:103DB0000102709002026419750986099709683C2E
:103DC00071058105910570F00E9427036093FF0142
:103DD00070930002809301029093020210930602F6
:103DE000109305027090FA0121E0472D62E080E116
:103DF0000E944A0B811108C097EEC91698E1D906B6
:103E00009FEFE906F10449F481E0870D8C3308F057
:103E100045C08093FA010E94BE0A7090FA0121E029
:103E2000472D62E08EE00E944A0B811108C0E5EB4D
:103E3000CE16EAE4DE06EFEFEE06F10441F48FEF72
:103E4000870D8C3370F58093FA010E94BE0A20E042
:103E500040E060E08FE00E944A0B811109C027EC2E
:103E6000C21628E3D2062FEFE206F10409F05ACF7A
:103E70000E94BE0A1092FB018091F90180931B02FF
:103E80008091FA0180931A0210921902D1CC1092FB
:103E9000F90118CF77E17093F9012FCF1092FA0151
:103EA000BACFFBE3F093FA01D0CF0E94F10CDECC45
:103EB0008F3450EB95075FEFA507B10519F40E9409
:103EC0000A15D4CC873668E996076FEFA607B105C7
:103ED00009F0ECC38091F80181110BC00E94C70B5F
:103EE00080E00E94F10C1092F70181E08093F801CC
:103EF000BDCC80E090E89093B4018093B30160E082
:103F000070E882E00E948D0B1092F801AFCC673E02
:103F100078418F4F910509F072CD21E0E21203C084
:103F20001092EA016CCDF092EA0169CD673E7841CA
:103F30008F4F910509F087CD61E0F61203C0109212
:103F4000E90181CDE092E9017ECD673E78418F4F56
:103F5000910509F09CCD21E0F21203C01092E80116
:103F600096CDE092E80193CD673E78418F4F910561
:103F700009F0B1CD61E0F61203C01092E701ABCDBC
:103F8000E092E701A8CD673E78418F4F910509F097
:103F9000C6CD21E0F21203C01092E601C0CDE0923E
:103FA000E601BDCDE092E501DECD71E0F712B8C3C8
:103FB000E090E4018E2D602F0E94E22A809303029C
:103FC00090930402F090E3018F2D0E94E22A8093E7
:103FD00005029093060210930702109308020E94B4
:103FE000000D609315027093160280931702909350
:103FF0001802673EE8E17E07EFEF8E07910539F47E
:1040000081E08E0D883170F01092E401D1CF653BD4
:10401000FAE47F07FFEF8F07910559F48FEF8E0DBC
:10402000883118F48093E401C3CF27E12093E401A1
:10403000BFCF653A3AE573073FEF8307910509F073
:1040400055C381E08F0D8C3318F48093E301B0CF1A
:104050001092E301ADCF8FEF8F0D8C33B0F35BE3A4
:104060005093E301A5CF1092E201D6C38735984A59
:10407000AF4FB10509F02BC49091EA018091E9019D
:10408000909F800D11248093CD011092E901109230
:10409000EA0188EC80937C0080917A0080688093AC
:1040A0007A0064E170E080E090E00E94F502809187
:1040B0007A00806480937A0080917A0086FDFCCF3C
:1040C000609178007091790090E080E00E94AE29C4
:1040D0002EEA37E242E953E40E94942826EF38E2C0
:1040E0004CE95FE30E9406296B017C0120E030E08F
:1040F000A9010E94602A20E030E040E05FE387FDF4
:1041000035C0C701B6010E9495280E9478296093A6
:10411000CC01862F602F0E94E22AF92E0E94E22A0B
:10412000E92E0E94000D6093150270931602809391
:104130001702909318021093080210930702E0925E
:104140000502F092060210930402109303026735F1
:10415000784A8F4F910529F78091CD01602F0E94F9
:10416000E22A9093E9018093EA01B1C3C701B60145
:104170000E949428CACF922F941B492F5985459F9E
:10418000040E40E0411D1124241B422F28C4262F79
:10419000231B3985239F020E20E0211D1124F21AD2
:1041A0004FC4242F2F19682F269F020E20E0211DB7
:1041B0001124421B242F50C4512C412C33C5188686
:1041C0001F8237C5A4E04A2E512C1C861B8636C59B
:1041D000F5E02F2E312C9101215031093A872987A2
:1041E000232B09F038C522242394312CE5E0F0E09C
:1041F000FE87ED8735C54E145F0459F40E94A82749
:10420000A50194010E94312869837A82F6E9FB8333
:1042100042C52F8138852E153F0559F40E94A827E5
:10422000A50194010E94312869837A8230E53B839D
:1042300032C56B857C856E157F0551F40E94A827D9
:10424000A50194010E94312869837A826B8223C57B
:104250002E143F0459F40E94A827A50194010E943E
:10426000312869837A8276E97B8315C589859A85A9
:104270008E159F0559F40E94A827A50194010E945C
:10428000312869837A8290E59B8305C5ED85FE859B
:10429000EE15FF0599F219821A821B82FCC4109256
:1042A000BA011092B9011FC5F70110821182128262
:1042B00038C5FBE3FF1508F4E5C58091E5018130C1
:1042C00009F03FC08091C1018823A1F00E9427031B
:1042D00020E137E240E050E00E946328672B682B22
:1042E000692B41F40E940A1561E070E080E090E0E3
:1042F0000E94F5029091F9018091E401981321C088
:104300009091FA018091E30198131BC08091FC0108
:10431000811117C08091F5019091F60190930101F0
:10432000809300010E94AE0B80E00E94F10C10927D
:10433000F7010E94C70B82E08093FC0181E080932B
:10434000C1018091FB01811114C08091C0018111D4
:1043500010C08091140281110CC04091FC01609149
:10436000FA018091F9019091E701911163C10E94D6
:10437000231580911402882309F467C0109210025B
:104380001092110210921202109213020E9427033F
:10439000C090FF01D0900002E0900102F090020274
:1043A0006C197D098E099F09683873418105910553
:1043B00008F43FC0109214028091F901F090FA01C4
:1043C0004091FC019091E70191113EC1602F0E9444
:1043D000E22A8093090290930A028F2D0E94E22A1A
:1043E00080930B0290930C02842F0E94E22A809308
:1043F0000D0290930E0236E0E32EF12C4EE0C42E17
:1044000042E0D42E80910302E3E0F2E091819193A7
:10441000CE16DF06D9F780930E0264E670E080E0E6
:1044200090E00E94F50271E0E71AF10859F70E9446
:104430001F0C8091CE018093EA014091FD016091B3
:10444000FE0180910F020E9423158091F9018230B4
:10445000D1F48091FA018E31B1F48091FC01811187
:1044600012C081E08093C0019091EA018091E9013E
:10447000909F800D11248093CD010E94260B1092F5
:10448000E9011092EA018091F901843099F4809158
:10449000FA018E3179F48091FC0181110BC01092E8
:1044A000C0018091CD01602F0E94E22A9093E90122
:1044B0008093EA018091C001882309F4B1C0809102
:1044C000BF01811165C00E94270324E6C22ED12CB2
:1044D000E12CF12CA70196010E946328CA01B901C1
:1044E0002AE030E040E050E00E9463286093080238
:1044F0000E942703A70196010E946328CA01B901FF
:104500002AE030E040E050E00E9463286093070218
:104510000E942703A70196010E946328CA01B901DE
:104520002AE030E040E050E00E94632860930602F9
:104530000E942703A70196010E946328CA01B901BE
:104540002AE030E040E050E00E94632860930502DA
:104550000E942703A70196010E946328CA01B9019E
:104560002AE030E040E050E00E94632860930402BB
:104570000E942703A70196010E946328CA01B9017E
:104580002AE030E040E050E00E946328609303029C
:104590000E94000D16161706180619065CF44091C5
:1045A000FC016091FA018091F9010E94231581E0DC
:1045B0008093BF018091BF01882391F18091BB015D
:1045C0009091BC01A091BD01B091BE010196A11DC9
:1045D000B11D8093BB019093BC01A093BD01B0932A
:1045E000BE014091FC016091FA018091F9010E94A5
:1045F00023158091BB019091BC01A091BD01B091A8
:10460000BE018135934CA105B10554F01092BB0158
:104610001092BC011092BD011092BE011092BF0118
:1046200080E090E0892B11F40C94451A0E94000060
:104630000C94431A3BE3341B432F5BE3561B652F5B
:1046400077E1781B872F93CE27E130E0B901681B13
:104650007109CB01EAE0F0E0BF010E94022B6093F8
:10466000090280930A022BE330E0C9018F199109F6
:10467000BF010E94022B60930B0280930C02C901C0
:10468000841B9109BF010E94022B60930D0280934D
:104690000E02B1CEFBE3FF1508F00FCE1092FA0127
:1046A000F090F901F394F092F901FFC38D35924A2D
:1046B000AF4FB10509F0DAC88091F5019091F6018C
:1046C00090930101809300010E94C4136091000146
:1046D000709101017093F6016093F501882309F44C
:1046E000C5C882E190E00E941C28C0C86F3E30E13E
:1046F00073073FEF8307910509F4ADCC673C78431E
:104700008F4F910509F054CC6091E40187E090E06F
:104710000E940E286091E30186E090E00E940E283E
:104720006091EA0185E090E00E940E286091E90125
:1047300084E090E00E940E286091E80183E090E020
:104740000E940E286091E70182E090E00E940E280E
:104750006091E50181E090E00E940E286091E60101
:1047600080E090E00E940E2820E040E060E080E1E0
:104770000E944A0B81110DC0809115029091160282
:10478000A0911702B0911802853A9A45AF4FB10532
:1047900031F51092E2018091E1012AE0722E780E4B
:1047A0007092E1018EE18093AD023FECE32E31E0A7
:1047B000F32E44EEC42E41E0D42E66246A9479820E
:1047C0006A826B82B701CE0101960E94590473E0A0
:1047D000E70EF11CCE14DF0491F70E94330320E0B2
:1047E00040E060E08EE00E944A0B81110DC0809194
:1047F000150290911602A0911702B09118028F3EF7
:104800009041AF4FB10571F48091E2018F5F853027
:1048100008F029CC8093E2018091E201811102C06D
:104820000E94260B8091150290911602A09117020A
:10483000B0911802853BFAE49F07FFEFAF07B1057F
:1048400009F014CC81E0809314028091EA018093F6
:10485000CE011092EA018091FD01602F0E94E22AB0
:104860009093090280930A028091FE010E94E22A3D
:1048700080930B0290930C0280910F020E94E22A17
:1048800090930D0280930E0296E0E92EF12C809118
:104890000302E3E0F2E09181919322E0EE30F2072F
:1048A000D1F780930E0264E670E080E090E00E9411
:1048B000F50231E0E31AF10851F70E9427036093F3
:1048C000FF01709300028093010290930202809195
:1048D000E201813009F019C18EE18093AD020E949E
:1048E0002703C090C801D090C901E090CA01F090A0
:1048F000CB016C197D098E099F0965317105810510
:10490000910508F446C10E9427036093C801709383
:10491000C9018093CA019093CB018FEC482E81E0AE
:10492000582E1F826090C6017090C701EBECF0E03A
:104930008491870D90E0FC01E553FF4F2490FC012A
:10494000E453FF4FE490ECECF0E08491870D90E0AD
:10495000FC01E553FF4F24912B87FC01E453FF4FEB
:10496000D490FF80F694C62CC6943C2C8F810E9474
:104970004A048987862D0E944A0430E83F0D5B85F2
:10498000E52FF0E0E553FF4FE491232F4C2DE2FD9E
:1049900002C02C2D432FE0FD4195E1FD2195259589
:1049A0004595421FE22DF0E0E553FF4FE4912F2D96
:1049B000E2FF02C02C2D3F2CE0FD2195E1FD31945A
:1049C000632D65952595261F24170CF0D4CB421B2B
:1049D0007985479F040E40E0411D1124420F20E8D5
:1049E0002C0DED2DF0E0E553FF4FE491522FE2FF47
:1049F00002C0532F322FE0FD3195E1FD51955595C1
:104A00003595351FEE2DF0E0E553FF4FE491E2FFC1
:104A100003C09F2DF22E292FE0FDF194E1FD219599
:104A20006F2D25956595621FF62E63170CF0AFCBA1
:104A3000361B7985379F030E30E0311D1124F30EAC
:104A40004F150CF0AECBF41A2F2D582F259F020EC8
:104A500020E0211D1124240F205C722F770F08F411
:104A60007FEFE72EF12C9701A5E1B0E00E948528A9
:104A7000A50194010E943128205B2983D70126EFEC
:104A80003FEF4FEF5FEF0E945028A50194010E9475
:104A9000312821503F4F4F4F5F4F2A839701A9EB99
:104AA000B0E00E948528A50194010E9431282A5B6C
:104AB0003F4F4F4F5F4F2B83BE016C5F7F4FCE0147
:104AC00001960E9459048C81F20180838D8181833B
:104AD0008E818283FF81F15FFF8323E0420E511CB0
:104AE000FA3509F01FCFC30144969093C701809314
:104AF000C6010E9433030E94000D6F3E70418F4F2C
:104B0000910519F482E08093E2018091E201823004
:104B100009F03FC02091B9013091BA012F5F3F4F9A
:104B20003093BA012093B9018091B5019091B601FB
:104B30000A969093B6018093B5012630310524F092
:104B40001092BA011092B9018F3F910529F024F01B
:104B50001092B6011092B5018091B50189838FEF53
:104B60008A838B838091B9019091BA01BC01660F51
:104B7000771F680F791F61537E4FCE0101960E9407
:104B800059040E94330362E370E080E090E00E94E9
:104B9000F5028091E201833009F094C08091B70161
:104BA0009091B801892BB9F48091B9019091BA0123
:104BB00001969093BA018093B901069709F581E0B7
:104BC00090E09093B8018093B70185E090E09093D6
:104BD000BA018093B9018091B7019091B801019712
:104BE00079F48091B9019091BA0101979093BA013B
:104BF0008093B901892B21F41092B8011092B7016A
:104C00002090B9013090BA0155E0251631040CF01E
:104C1000D3CA21016FEF461A560A75E047165104B0
:104C200009F4CDCAC201019698878F83059709F4CC
:104C3000C9CAEF81F8853196FC87EB8712141304FB
:104C40000CF0C6CAF1E02F1A310809F0C4CA65E0B9
:104C500070E07A87698789859A8501979E878D8715
:104C60006FECC62E61E0D62EF12CE12C77247A94DD
:104C700074E1672E8091B9019091BA018E159F055C
:104C800009F0B9CA0E94A827A50194010E94312801
:104C900069837A827B82B601CE0101960E94590413
:104CA000FFEFEF1AFF0A23E0C20ED11C36E0E31635
:104CB000F10401F70E94330364E670E080E090E0C5
:104CC0000E94F5028091E2018430E9F58091B901FA
:104CD0009091BA010196873091050CF0E0CA90934B
:104CE000BA018093B9015FECE52E51E0F52ED12C8D
:104CF000C12C77247A948091B9019091BA018C15D6
:104D00009D0509F0D1CA0E94A827A50194010E941F
:104D1000312869837A827B82B701CE0101960E9495
:104D20005904FFEFCF1ADF0A23E0E20EF11C36E050
:104D3000C316D10401F70E94330364E670E080E0FB
:104D400090E00E94F5028091FA0165E00E94E22A5B
:104D5000911106C08091FC01811102C00E941F0CBC
:104D60000E942703C090C201D090C301E090C4010B
:104D7000F090C5016C197D098E099F09683E73404A
:104D80008105910508F499CA8091FB01811195CAAA
:104D90000E9427036093C2017093C3018093C401F2
:104DA0009093C501E090FC01E394E092FC018091B6
:104DB000E901813041F58E2D6EE10E94E22AF92E43
:104DC000911121C0F0920302F0920402F0920502C8
:104DD000F0920602F0920702F092080264E170E09D
:104DE00080E090E00E94F502F3946AE0F612EACFC8
:104DF00010920702109208024E2D6091FA018091E4
:104E0000F9010E942315E090EA01F090FC0171E0A5
:104E1000E71210C08091140281110CC085E00E943D
:104E2000CF0A8F2D602F0E94E22A911103C084E0E7
:104E30000E94CF0A8091E801813011F40E94E90AB2
:104E40008BE38F1508F039CA1092FC01F090FA013B
:104E5000F394F092FA0191E0E9121CCC80911402D3
:104E6000811127CA83E00E94CF0A8F2D602F0E94F4
:104E7000E22A91111ECA82E00E94CF0AEBE3EF15ED
:104E800008F01BCA1092FA01F090F901F394F09225
:104E9000F90181E00E94CF0A8F2D602F0E94E22A43
:104EA000911103C080E00E94CF0A27E12F1508F07E
:104EB00004CA1092F90101CA8F929F92AF92BF92D9
:104EC000CF92DF92EF92FF92CF93DF93EC01688154
:104ED00079818A819B81611571058105910521F494
:104EE00064E279ED8BE597E02DE133EF41E050E0AE
:104EF0000E94312849015A019B01AC01A7EAB1E4A3
:104F00000E9450286B017C01ACEEB4EFA501940126
:104F10000E945E28C60ED71EE81EF91EF7FE06C0C8
:104F200081E0C81AD108E10880E8F80AC882D9826D
:104F3000EA82FB82C701B6019F77DF91CF91FF9094
:104F4000EF90DF90CF90BF90AF909F908F9008959B
:104F50008F929F92AF92BF92CF92DF92EF92FF9289
:104F60006091030170910401809105019091060107
:104F7000611571058105910521F464E279ED8BE5F8
:104F800097E02DE133EF41E050E00E9431284901E4
:104F90005A019B01AC01A7EAB1E40E9450286B01C1
:104FA0007C01ACEEB4EFA50194010E945E28C60E10
:104FB000D71EE81EF91EF7FE06C081E0C81AD10808
:104FC000E10880E8F80AC0920301D0920401E0925F
:104FD0000501F0920601C701B6019F77FF90EF909F
:104FE000DF90CF90BF90AF909F908F900895609387
:104FF00003017093040180930501909306010895C5
:10500000F999FECF92BD81BDF89A992780B5089590
:10501000A8E1B0E042E050E00C942328262FF99953
:10502000FECF1FBA92BD81BD20BD0FB6F894FA9A8B
:10503000F99A0FBE019608950E940E28272F0C940E
:105040000F28DC01CB01FC01F999FECF06C0F2BDAF
:10505000E1BDF89A319600B40D9241505040B8F736
:105060000895052E97FB1EF400940E94482857FDD2
:1050700007D00E94632807FC03D04EF40C94482804
:1050800050954095309521953F4F4F4F5F4F089574
:1050900090958095709561957F4F8F4F9F4F0895A4
:1050A0000E948528A59F900DB49F900DA49F800D10
:1050B000911D11240895B7FF0C9450280E94502888
:1050C000821B930B0895A1E21A2EAA1BBB1BFD01A4
:1050D0000DC0AA1FBB1FEE1FFF1FA217B307E407D7
:1050E000F50720F0A21BB30BE40BF50B661F771F2F
:1050F000881F991F1A9469F760957095809590950F
:105100009B01AC01BD01CF010895A29FB001B39FE7
:10511000C001A39F700D811D1124911DB29F700DC0
:10512000811D1124911D08955058BB27AA270E9464
:10513000AC280C94262A0E94182A38F00E941F2AB4
:1051400020F039F49F3F19F426F40C94152A0EF43C
:10515000E095E7FB0C940F2AE92F0E94372A58F3B9
:10516000BA17620773078407950720F079F4A6F54C
:105170000C94592A0EF4E0950B2EBA2FA02D0B019A
:10518000B90190010C01CA01A0011124FF27591B8C
:1051900099F0593F50F4503E68F11A16F040A22F92
:1051A000232F342F4427585FF3CF46953795279503
:1051B000A795F0405395C9F77EF41F16BA0B620B02
:1051C000730B840BBAF09150A1F0FF0FBB1F661F49
:1051D000771F881FC2F70EC0BA0F621F731F841F8C
:1051E00048F4879577956795B795F7959E3F08F0B2
:1051F000B0CF9395880F08F09927EE0F9795879574
:1052000008950E94EB2908F481E008950E941A296C
:105210000C94262A0E941F2A58F00E94182A40F057
:1052200029F45F3F29F00C940F2A51110C945A2A4B
:105230000C94152A0E94372A68F39923B1F3552359
:1052400091F3951B550BBB27AA2762177307840799
:1052500038F09F5F5F4F220F331F441FAA1FA9F32F
:1052600035D00E2E3AF0E0E832D091505040E6951D
:10527000001CCAF72BD0FE2F29D0660F771F881F7E
:10528000BB1F261737074807AB07B0E809F0BB0B71
:10529000802DBF01FF2793585F4F3AF09E3F510585
:1052A00078F00C940F2A0C945A2A5F3FE4F3983E4E
:1052B000D4F3869577956795B795F7959F5FC9F76E
:1052C000880F911D9695879597F90895E1E0660FEF
:1052D000771F881FBB1F621773078407BA0720F068
:1052E000621B730B840BBA0BEE1F88F7E0950895D1
:1052F0000E947F296894B1110C945A2A08950E9443
:105300003F2A88F09F5798F0B92F9927B751B0F0EE
:10531000E1F0660F771F881F991F1AF0BA95C9F739
:1053200014C0B13091F00E94592AB1E008950C9454
:10533000592A672F782F8827B85F39F0B93FCCF307
:10534000869577956795B395D9F73EF490958095B6
:10535000709561957F4F8F4F9F4F0895E89409C0D6
:1053600097FB3EF490958095709561957F4F8F4F98
:105370009F4F9923A9F0F92F96E9BB279395F695AE
:10538000879577956795B795F111F8CFFAF4BB0F2C
:1053900011F460FF1BC06F5F7F4F8F4F9F4F16C090
:1053A000882311F096E911C0772321F09EE8872F1A
:1053B000762F05C0662371F096E8862F70E060E0D6
:1053C0002AF09A95660F771F881FDAF7880F96954F
:1053D000879597F90895990F0008550FAA0BE0E8F3
:1053E000FEEF16161706E807F907C0F012161306A7
:1053F000E407F50798F0621B730B840B950B39F4E7
:105400000A2661F0232B242B252B21F408950A264C
:1054100009F4A140A6958FEF811D811D089597F98C
:105420009F6780E870E060E008959FEF80EC08954A
:1054300000240A9416161706180609060895002473
:105440000A9412161306140605060895092E0394ED
:10545000000C11F4882352F0BB0F40F4BF2B11F461
:1054600060FF04C06F5F7F4F8F4F9F4F089557FDC0
:105470009058440F551F59F05F3F71F04795880FC2
:1054800097FB991F61F09F3F79F087950895121659
:1054900013061406551FF2CF4695F1DF08C0161605
:1054A00017061806991FF1CF8695710561050894B6
:1054B0000895E894BB2766277727CB0197F90895CD
:1054C0000E94EB2908F48FEF08950E94782A0C942B
:1054D000262A0E94182A38F00E941F2A20F09523BD
:1054E00011F00C940F2A0C94152A11240C945A2AAA
:1054F0000E94372A70F3959FC1F3950F50E0551F16
:10550000629FF001729FBB27F00DB11D639FAA2718
:10551000F00DB11DAA1F649F6627B00DA11D661F67
:10552000829F2227B00DA11D621F739FB00DA11D88
:10553000621F839FA00D611D221F749F3327A00D42
:10554000611D231F849F600D211D822F762F6A2FDE
:1055500011249F5750409AF0F1F088234AF0EE0F43
:10556000FF1FBB1F661F771F881F91505040A9F770
:105570009E3F510580F00C940F2A0C945A2A5F3FED
:10558000E4F3983ED4F3869577956795B795F795AC
:10559000E7959F5FC1F7FE2B880F911D9695879524
:1055A00097F90895DB018F939F930E945028BF9134
:1055B000AF91A29F800D911DA39F900DB29F900D62
:1055C00011240895991B79E004C0991F961708F0DB
:1055D000961B881F7A95C9F780950895AA1BBB1B57
:1055E00051E107C0AA1FBB1FA617B70710F0A61BE3
:1055F000B70B881F991F5A95A9F780959095BC0104
:10560000CD01089597FB072E16F4009407D077FD7F
:1056100009D00E94EE2A07FC05D03EF490958195B2
:105620009F4F0895709561957F4F08950E9485283A
:10563000B7FF0895821B930B0895002E083090F059
:10564000982F872F762F652F542F432F322F222705
:105650000850F4CF220F331F441F551F661F771FBA
:10566000881F991F0A95B2F7002D089597FD109491
:10567000002E083098F00850232F342F452F562F36
:10568000672F782F892F912DF4CF159497958795B3
:105690007795679557954795379527950A95AAF772
:1056A0001124002D0895EE0FFF1F0590F491E02DB9
:1056B000099481E090E0F8940C945E2BF894FFCF6D
:1056C000F50301010000000008020A0109030B04B0
:1056D0000C000000006E156E156E15FB0BF70BF439
:1056E0000B000000007B0A370A350AFB0BF70BBCE6
:1056F0000154070000000058062B06140701062479
:065700000611060206007E
:00000001FF
